:100000000C9456040C9473040C9473040C947304B1
:100010000C9473040C9473040C9473040C94730484
:100020000C9473040C9473040C9473040C94730474
:100030000C9473040C9473040C9473040C94730464
:100040000C9475040C9473040C94EC1A0C94E31A3D
:100050000C9473040C9473040C9473040C94730444
:100060000C9473040C9473040C9473040C94730434
:100070000C9473040C9473040C9473040C94730424
:100080000C9473040C9473040C9473043A0AEE0CED
:10009000420A5B0A790AEE0CEE0CEE0CEE0CEE0C4A
:1000A000EE0CEE0CEE0CEE0CEE0CEE0C8E098B0949
:1000B000880994099109EE0CEE0CEE0CEE0C270C5D
:1000C000EE0CEE0CEE0CEE0CC604EE0C7B09EE0C06
:1000D000EE0C7209B20CE50A9D0BEE0CA90CEE0CAD
:1000E000EE0CAC0CEE0CEE0CEE0CAF0CEE0CB00A01
:1000F0006909190BEE0CEE0CEE0CEE0CEE0CEE0C8E
:10010000EE0CEE0CEE0C920AEE0C330A2D0CEE0CFB
:10011000E10B0105EE0C2D0C360CC90CEE0CEE0CAF
:10012000BB0CC00CEE0C590BEC0CEE0CEE0C9B094E
:10013000EE0CEE0CEE0CEE0CEE0CC50C0852573F1C
:100140009F5A49CBA5620F76C76913F27E6F500D97
:100150000175360B617A2AAAAB7E0000007F000091
:1001600000000A0D53525831204578656375746953
:1001700076652076657273696F6E20312E30000AC5
:100180000D3D3D3D3D3D3D3D3D3D3D3D3D3D3D3DCF
:100190003D3D3D3D3D3D3D3D3D3D3D3D3D3D3D3D8F
:1001A0003D3D3D3D3D3D3D3D000A0D517569747439
:1001B000696E672E2E2E0A0D000A0D5265626F6F52
:1001C00074696E672E2E2E000A0D456E74657220BE
:1001D000706F7274206C65747465723A20000A0D39
:1001E000504F5254000937363534333231300A0D0E
:1001F0000909000A0D2D2D2D2D2D2D2D2D2D2D2DE7
:100200002D2D2D2D2D2D2D2D2D2D2D2D2D2D2D2D1E
:100210002D2D2D2D2D2D2D2D2D2D2D000A0D426531
:10022000686176696F757209456E61626C65640913
:10023000537461747573095072696F7269747909C6
:100240004F757470757409547970650A0D3D3D3DA4
:100250003D3D3D3D3D3D093D3D3D3D3D3D3D093D36
:100260003D3D3D3D3D093D3D3D3D3D3D3D3D093D26
:100270003D3D3D3D3D093D3D3D3D0A0D000A0D45DD
:100280006E746572204932432061646472657373D1
:100290003A20000A0D456E74657220656C656D65C7
:1002A0006E743A20000A0D456E74657220646174A4
:1002B000613A20000A0D4C696E652053656E736FBC
:1002C00072733A20000A0D4552524F523A20000AEA
:1002D0000D43617274657369616E20506F73697448
:1002E000696F6E3A20000A0D475032443132207255
:1002F000656164696E67733A000A0D4944090950E3
:100300006172616D6574657209090956616C756584
:100310000A0D2D2D09092D2D2D2D2D2D2D2D2D09BC
:1003200009092D2D2D2D2D000A0D30310909466F9B
:100330006C6C6F77205020636F65666669636965D2
:100340006E740909000A0D30320909466F6C6C6F32
:1003500077204420636F656666696369656E74091A
:1003600009000A0D303309094D6F746F7220502057
:10037000636F656666696369656E740909000A0DD5
:10038000303409094D6F746F72204920636F6566C0
:1003900066696369656E740909000A0D30350909DB
:1003A0004D6F746F72204420636F65666669636980
:1003B000656E740909000A0D303609094C696E65CD
:1003C0002053656E736F72205468726573686F6C2A
:1003D000640909000A0D3037090953434D20457857
:1003E000706F7375726520486967680909000A0DA6
:1003F0003038090953434D204578706F7375726525
:10040000204C6F770909000A0D3039090953434D13
:10041000205468726573686F6C64090909000A0DDD
:100420003130090953434D204D696E696D756D205A
:1004300053697A65205468726573686F6C6409004B
:100440000A0D454449543A20456E74657220506146
:1004500072616D6574657220494420283020746F84
:100460002071756974293A0A0D000A0D0909093DC0
:100470003D3D3D3D3D3D3D3D2048656C70203D3D51
:100480003D3D3D3D3D3D3D000A0D64202D20447520
:100490006D70207374617475730909090972202DD8
:1004A0002052656164206120706F7274000A0D78BB
:1004B000202D2053434D204175746F2D63616C696D
:1004C00062726174696F6E09096F202D2052657325
:1004D0006574204F646F6D65747279000A0D532046
:1004E0002D2053746F70206D6F746F72730909093A
:1004F0000941202D20526F74617465204C6566742B
:10050000000A0D44202D20526F74617465205269D9
:1005100067687409090931202D20466F727761726E
:1005200064204C6F77000A0D32202D20466F7277C1
:10053000617264204D656469756D09090933202D68
:1005400020466F72776172642048696768000A0DFF
:1005500034202D204261636B77617264204C6F7789
:1005600009090935202D204261636B77617264208F
:100570004D656469756D000A0D52202D20526F740F
:10058000617465204162732F52656C090909462028
:100590002D2054726176656C2064697374616E639A
:1005A000652028636D29000A0D54202D20466F6CAC
:1005B0006C6F772057616C6C0909090947202D2061
:1005C000476F20417420636F6F7264696E61746558
:1005D000000A0D6E202D20416C69676E20772F2058
:1005E00057616C6C2F446F6F7209090968202D20C8
:1005F000476F20486F6D652066726F6D20726F6F58
:100600006D206E000A0D6B202D206B696C6C2050E4
:100610004C414E4E45520909096C202D2077616BE3
:100620006520757020504C414E4E4552000A0D66B3
:10063000202D20546F67676C6520464F4C4C4F57F8
:1006400020646562756709090961202D20546F6770
:10065000676C6520415242495452415445206465BB
:10066000627567000A0D4C202D2052656C6F616425
:1006700020506172616D65746572205461626C65B1
:10068000090949202D2052652D496E697420506159
:1006900072616D65746572205461626C65000A0D4B
:1006A00050202D2044756D7020506172616D65740D
:1006B0006572205461626C65090945202D204564EE
:1006C000697420506172616D657465722054616255
:1006D0006C65000A0D21202D20536F6674776172BE
:1006E000652052657365742121212109090967205C
:1006F0002D2044756D702053434D207265676973DA
:100700007465727300455845430041564F49440093
:10071000464F525741524400474F5F41540045589D
:1007200054494E475549534800414C49474E0052A1
:100730004F414D00524F544154450053454152439F
:100740004800464F4C4C4F5700350584047804044C
:10075000E1058A15E805022E06E10F8E02058C05DB
:1007600050128202058403100E2D0405D4021B0FC3
:10077000E80205CC04C90E3C050339033615D7043D
:10078000057D0293133A03057304040D210404C587
:1007900003E610E20505496C6C6567616C20526FD9
:1007A0006F6D202300FFFFFFFFFFFFFFFFFFFFFF35
:1007B000FFFFFFFFFFFFFFFFFFFFFFFFFFFFFFFF49
:1007C000FFFFFFFFFFFFFFFFFFFFFFFFFFFFFFFF39
:1007D000FFFFFFFFFF3C3A393837363534333231CB
:1007E000302F2E2E2D2C2B2B2A2929282727262661
:1007F000252524242323222221212120201F1F1FDD
:100800001E1E1E1D1D1D1C1C1C1B1B1B1B1A1A1A29
:100810001A1919191918181818171717171716165B
:10082000161616151515151515141414141414137D
:100830001313131313131212121212121212111194
:1008400011111111111111101010101010101010A1
:100850000F0F0F0F0F0F0F0F0F0F0F0E0E0E0E0EAD
:100860000E0E0E0E0E0E0E0E0D0D0D0D0D0D0D0DB0
:100870000D0D0D0D0D0D0C0C0C0C0C0C0C0C0C0CB2
:100880000C0C0C0C0C0C0B0B0B0B0B0B0B0B0B0BB2
:100890000B0B0B0B0B0B0B0B0B0B0A0A0A0A0A0AAE
:1008A0000A0A0A0A99067B1DB006010011241FBE20
:1008B000CFEFD0E1DEBFCDBF11E0A0E0B1E0E8EFC7
:1008C000FFE400E00BBF02C007900D92A030B1071B
:1008D000D9F716E0A0E0B1E001C01D92A73CB10736
:1008E000E1F70C94B3160C9400000E94F12286EFFD
:1008F00082BF0E9496240E94B7200B9B02C0C19A1F
:1009000001C0C1980E943D23FF24F0921F0181E0A5
:10091000809328010E94DB1A8036E1F710922401AF
:1009200010922301109226011092250181E08093FC
:1009300021016BE171E084E794E00E94DA248BE10D
:1009400091E00E94D9231092000182E691E00E947A
:10095000F91A8FE791E00E94F91A0E94F01B8EE3CA
:100960000E94C51A0E940B1B9927AA27BB27FC01CE
:10097000B197E835F10510F00C94EE0CEA5BFF4FEF
:10098000EE0FFF1F0590F491E02D09948AE694E0A4
:100990000E94F91A88E894E00E94F91A8DEA94E01E
:1009A0000E94F91A8CED94E00E94F91A81E095E01A
:1009B0000E94F91A86E295E00E94F91A8EE495E009
:1009C0000E94F91A87E795E00E94F91A87EA95E0F4
:1009D0000E94F91A81ED95E00E94F91A84E096E0F0
:1009E0000E94F91A8DE296E00E94F91A84E696E0D8
:1009F0000E94F91A8EE996E00E94F91A83ED96E0BA
:100A000036C58FE791E00E94F91A8FEC92E00E94C0
:100A1000F91A88E50E94C51A8DE30E94C51A8091D3
:100A20002A0290912B020E94B31C80E20E94C51AF8
:100A300089E50E94C51A8DE30E94C51A80912C0297
:100A400090912D020E94B31C80E20E94C51A80E49E
:100A50000E94C51A8DE30E94C51A80912E029091C2
:100A60002F020E94B31C83EF91E00E94F91A8CE1DF
:100A700092E00E94F91A85E097E00E94F91A89E055
:100A80000E94C51A89E00E94C51A8091C703882375
:100A900011F081E301C080E30E94C51A89E00E9441
:100AA000C51A8091C803882311F081E301C080E357
:100AB0000E94C51A89E00E94C51A8091C9030E944C
:100AC000F91C89E00E94C51A89E00E94C51A80912C
:100AD000CA039091CB030E94B31C8CE20E94C51AFA
:100AE0008091CC039091CD030E94B31C89E00E94B9
:100AF000C51A8091CF03813011F481E401C082E5F1
:100B00000E94C51A0E94F01B82E497E00E94F91A25
:100B100089E00E94C51A89E00E94C51A8091D0031D
:100B2000882311F081E301C080E30E94C51A89E0A7
:100B30000E94C51A8091D103882311F081E301C07E
:100B400080E30E94C51A89E00E94C51A8091D203F1
:100B50000E94F91C89E00E94C51A89E00E94C51A0A
:100B60008091D3039091D4030E94B31C8CE20E9425
:100B7000C51A8091D5039091D6030E94B31C89E0D9
:100B80000E94C51A8091D803813011F481E401C01C
:100B900082E50E94C51A0E94F01B8AE097E00E943D
:100BA000F91A89E00E94C51A89E00E94C51A80914D
:100BB000F403882311F081E301C080E30E94C51A89
:100BC00089E00E94C51A8091F503882311F081E322
:100BD00001C080E30E94C51A89E00E94C51A809175
:100BE000F6030E94F91C89E00E94C51A89E00E9460
:100BF000C51A8091F7039091F8030E94B31C8CE210
:100C00000E94C51A8091F9039091FA030E94B31CC7
:100C100089E00E94C51A8091FC03813011F481E4BF
:100C200001C082E50E94C51A0E94F01B88E197E08E
:100C30000E94F91A89E00E94C51A89E00E94C51A2B
:100C40008091EB03882311F081E301C080E30E94CF
:100C5000C51A89E00E94C51A8091EC03882311F01F
:100C600081E301C080E30E94C51A89E00E94C51A91
:100C70008091ED030E94F91C89E00E94C51A89E069
:100C80000E94C51A8091EE039091EF030E94B31C5D
:100C90008CE20E94C51A8091F0039091F1030E94AA
:100CA000B31C89E00E94C51A8091F303813011F4CE
:100CB00081E401C082E50E94C51A0E94F01B8EE10A
:100CC00097E00E94F91A89E00E94C51A80910604F3
:100CD000882311F081E301C080E30E94C51A89E0F6
:100CE0000E94C51A80910704882311F081E301C096
:100CF00080E30E94C51A89E00E94C51A8091080409
:100D00000E94F91C89E00E94C51A89E00E94C51A58
:100D10008091090490910A040E94B31C8CE20E9405
:100D2000C51A80910B0490910C040E94B31C89E0B9
:100D30000E94C51A80910E04813011F481E401C033
:100D400082E50E94C51A0E94F01B84E397E00E948E
:100D5000F91A89E00E94C51A89E00E94C51A80919B
:100D6000D903882311F081E301C080E30E94C51AF2
:100D700089E00E94C51A8091DA03882311F081E38B
:100D800001C080E30E94C51A89E00E94C51A8091C3
:100D9000DB030E94F91C89E00E94C51A89E00E94C9
:100DA000C51A8091DC039091DD030E94B31C8CE294
:100DB0000E94C51A8091DE039091DF030E94B31C4C
:100DC00089E00E94C51A8091E103813011F481E429
:100DD00001C082E50E94C51A0E94F01B89E297E0DB
:100DE0000E94F91A89E00E94C51A89E00E94C51A7A
:100DF00080911804882311F081E301C080E30E94F0
:100E0000C51A89E00E94C51A80911904882311F03F
:100E100081E301C080E30E94C51A89E00E94C51ADF
:100E200080911A040E94F91C89E00E94C51A89E089
:100E30000E94C51A80911B0490911C040E94B31C4F
:100E40008CE20E94C51A80911D0490911E040E949C
:100E5000B31C89E00E94C51A80912004813011F4EE
:100E600081E401C082E50E94C51A0E94F01B80E166
:100E700097E00E94F91A89E00E94C51A89E00E9451
:100E8000C51A8091E203882311F081E301C080E359
:100E90000E94C51A89E00E94C51A8091E303882345
:100EA00011F081E301C080E30E94C51A89E00E942D
:100EB000C51A8091E4030E94F91C89E00E94C51ABA
:100EC00089E00E94C51A8091E5039091E6030E9493
:100ED000B31C8CE20E94C51A8091E7039091E8034D
:100EE0000E94B31C89E00E94C51A8091EA038130F8
:100EF00011F481E401C082E50E94C51A0E94F01B32
:100F00008BE397E00E94F91A89E00E94C51A89E0F4
:100F10000E94C51A80910F04882311F081E301C05B
:100F200080E30E94C51A89E00E94C51A80911004CE
:100F3000882311F081E301C080E30E94C51A89E093
:100F40000E94C51A809111040E94F91C89E00E9438
:100F5000C51A89E00E94C51A809112049091130469
:100F60000E94B31C8CE20E94C51A809114049091D7
:100F700015040E94B31C89E00E94C51A80911704D1
:100F8000813011F481E401C082E50E94C51A0E94FB
:100F9000F01B8FE297E00E94F91A89E00E94C51ABF
:100FA00089E00E94C51A8091FD03882311F081E336
:100FB00001C080E30E94C51A89E00E94C51A809191
:100FC000FE03882311F081E301C080E30E94C51A6B
:100FD00089E00E94C51A8091FF030E94F91C89E0F4
:100FE0000E94C51A89E00E94C51A80910004909160
:100FF00001040E94B31C8CE20E94C51A8091020475
:10100000909103040E94B31C89E00E94C51A80914C
:101010000504813011F481E401C082E50E94C51A03
:1010200083EF91E00E94F91A0E94F01B80E50E9474
:10103000C51A8DE30E94C51A8091DC026AE00E9405
:10104000A5270E949B1C8EE20E94C51A8091DC029B
:101050006AE00E94A527892F0E94F91C80E20E9465
:10106000C51A89E40E94C51A8DE30E94C51A8091B1
:10107000DD026AE00E94A5270E949B1C8EE20E946E
:10108000C51A8091DD026AE00E94A527892F0E947F
:10109000F91C80E20E94C51A84E40E94C51A8DE3FF
:1010A0000E94C51A8091DE026AE00E94A5270E9474
:1010B0009B1C8EE20E94C51A8091DE026AE00E94AB
:1010C000A527892F0E94F91C0E94F01B80E70E942F
:1010D000C51A8DE30E94C51A8091DA026AE00E9467
:1010E000A5270E949B1C8EE20E94C51A8091DA02FD
:1010F0006AE00E94A527892F0E94F91C80E20E94C5
:10110000C51A84E60E94C51A8DE30E94C51A809113
:10111000DB026AE00E94A5270E949B1C8EE20E94CF
:10112000C51A8091DB026AE00E94A527892F0E94E0
:10113000F91C83EF91E00E94F91A84EB92E00E947F
:10114000F91A8CE40E94C51A8AE30E94C51A86E047
:101150000E94C319082F8091DF02801710F481E3E9
:1011600001C080E30E94C51A80E20E94C51A88E28D
:101170000E94C51A802F0E94F91C89E20E94C51A9C
:1011800080E20E94C51A82E50E94C51A8AE30E9485
:10119000C51A87E00E94C319082F8091DF028017CB
:1011A00010F481E301C080E30E94C51A80E20E942E
:1011B000C51A88E20E94C51A802F0E94F91C89E294
:1011C0000E94C51A83EF91E00E94F91A86EE92E020
:1011D0000E94F91A89E00E94C51A89E00E94C51A86
:1011E00080E00E94DF190E94F91C0E94F01B89E038
:1011F0000E94C51A89E00E94C51A89E00E94C51A9A
:1012000081E00E94DF190E94F91C89E00E94C51A42
:1012100089E00E94C51A83E00E94DF190E94F91C30
:101220000E94F01B89E00E94C51A89E00E94C51A3D
:1012300089E00E94C51A82E00E94DF190E94F91C11
:1012400089E00E94C51A89E00E94C51A84E00E94C4
:10125000DF190E94F91C83EF91E00E94F91A0E94A5
:10126000F01B83E50E94C51A83E40E94C51A8DE431
:101270000E94C51A8AE30E94C51A80E20E94C51A1C
:1012800062E080EB0E9476218823A1F088E20E9430
:10129000C51A64E080EB0E9476210E94F91C8CE262
:1012A0000E94C51A65E080EB0E9476210E94F91C1D
:1012B00089E20AC08EE40E94C51A8FE60E94C51A10
:1012C0008EE60E94C51A85E60E94C51A8FE791E056
:1012D000CEC0109224011092230110922601109288
:1012E00025016FC38CEE9FEF90932601809325011B
:1012F00084E190E008C084E190E09093260180931F
:1013000025018CEE9FEF909324018093230159C314
:1013100084E290E00BC086E190E008C08EE090E0AF
:1013200005C08AEE9FEF02C082EF9FEF90932601E7
:1013300080932501E8CF88EC91E00E94F91A0E9481
:101340000B1B682F77276534710509F477C0663465
:1013500071059CF462347105C1F16334710524F4A4
:1013600061347105F9F03AC36334710509F440C082
:101370006434710509F44FC031C363367105C1F19E
:10138000643671053CF46136710561F062367105B1
:10139000E1F024C364367105F1F16536710509F495
:1013A0004DC01CC38EED91E00E94F91A81E40E94A9
:1013B000C51A8DE30E94C51A89B30E94A61B85EE4B
:1013C00091E00E94F91A89B34BC08EED91E00E9422
:1013D000F91A82E40E94C51A8DE30E94C51A86B3E9
:1013E0000E94A61B85EE91E00E94F91A86B338C0D0
:1013F0008EED91E00E94F91A83E40E94C51A8DE3F4
:101400000E94C51A85B30E94A61B85EE91E00E943A
:10141000F91A85B325C08EED91E00E94F91A84E493
:101420000E94C51A8DE30E94C51A80B30E94A61BB4
:1014300085EE91E00E94F91A80B312C08EED91E022
:101440000E94F91A85E40E94C51A8DE30E94C51A0C
:1014500081B10E94A61B85EE91E00E94F91A81B12C
:101460000E94E31CBBC231E0F32E89EA91E00E94A6
:10147000F91AB4C289EB91E00E94F91AF8940E941B
:101480000000ACC28DE792E00E94F91A0E94191B7D
:10149000082F0E94F01B83E992E00E94F91A0E9433
:1014A000191BC82F0E94F01B6C2F802F0E947621E1
:1014B0000E94A61B93C28DE792E00E94F91A0E9437
:1014C000191B182F0E94F01B83E992E00E94F91A61
:1014D0000E94191B082F0E94F01B85EA92E00E94CF
:1014E000F91A0E94191B482F602F812F0E94CC21CE
:1014F00075C28DE792E00E94F91A0E94191B082F0D
:101500000E94F01B83E992E00E94F91A0E94191BC5
:10151000C82F0E94F01B6C2F802F0E9420220E9457
:10152000961B5CC28DE792E00E94F91A0E94191B7B
:10153000182F0E94F01B83E992E00E94F91A0E9482
:10154000191B082F0E94F01B85EA92E00E94F91AED
:101550000E94151BAC01602F812F0E945E223EC2AB
:101560008AE30E94C51A0E94DB1A082F813411F009
:101570008235C9F7802F0E94C51A023519F41092DE
:10158000090103C081E08093090110920A018AE3F6
:101590000E94C51A0E94211D9093080180930701A3
:1015A000109221016BE171E084E794E00E94DA245B
:1015B0008BE191E00E94D92363E071E083E995E03B
:1015C0000E94DA2483E091E0F9C08AE30E94C51A00
:1015D0000E94211D9093110180931001109212011D
:1015E000109221016BE171E084E794E00E94DA241B
:1015F0008BE191E00E94D9236CE071E08EE792E0EC
:101600000E94DA248CE091E00E94D92381E080934B
:1016100021016BE171E084E794E00E94DA248BE120
:1016200091E00E94D9238DE30E94C51A8091130195
:101630008DC18AE30E94C51A0E94DB1A082F8C34E0
:1016400011F08235C9F7802F0E94C51A1092190136
:101650000C3419F41092180103C081E08093180132
:10166000109221016BE171E084E794E00E94DA249A
:101670008BE191E00E94D92364E171E08DEC94E06C
:101680000E94DA2484E191E00E94D92381E08093D2
:1016900021016BE171E084E794E00E94DA248BE1A0
:1016A00091E00E94D9238DE30E94C51A80911A010E
:1016B0004DC18AE30E94C51A0E94DB1A082F8C34A0
:1016C00021F0823511F08434B9F7802F0E94C51AB9
:1016D0000C3419F41092420107C0043411F482E072
:1016E00001C081E080934201109221016BE171E021
:1016F00084E794E00E94DA248BE191E00E94D923F0
:101700006EE371E08DED94E00E94DA248EE391E0C7
:101710000E94D92381E0809321016BE171E084E78D
:1017200094E00E94DA248BE191E00E94D9238DE3BA
:101730000E94C51A8091430109C180E20E94C51A26
:1017400088E50E94C51A8AE30E94C51A0E94211DDD
:1017500090932E0180932D0180E20E94C51A89E5A5
:101760000E94C51A8AE30E94C51A0E94211D909307
:10177000300180932F0180E20E94C51A80E40E940C
:10178000C51A8AE30E94C51A0E94001C9093320178
:1017900080933101109221016BE171E084E794E0C4
:1017A0000E94DA248BE191E00E94D92369E271E082
:1017B00084EE92E00E94DA2489E291E00E94D9232B
:1017C000FDC08AE30E94C51A0E94DB1A082F8C34E0
:1017D00011F08235C9F7802F0E94C51A0C3419F414
:1017E00010923D0103C081E080933D0110922101E0
:1017F0006BE171E084E794E00E94DA248BE191E0F0
:101800000E94D92368E371E085ED92E00E94DA241A
:1018100088E391E00E94D92380913C01813051F40A
:1018200063E371E080E493E00E94DA2483E391E0D3
:101830000E94D9238DE30E94C51A80913C0181301A
:1018400011F481E301C080E30E94C51AB7C01A9B5E
:1018500002C01A98C3C01A9AC1C090E080910101D9
:10186000882309F491E090930101B8C000E00E9440
:10187000F01B802F0E94F91C8AE30E94C51A025FA8
:10188000602F80EB0E9476210E94A61B0D500E3027
:1018900070F30E94F01B81E40E94C51A8AE30E9443
:1018A000C51A66E080EB0E9476210E94F91C0E9416
:1018B000F01B84E50E94C51A8AE30E94C51A67E0FE
:1018C00080EB0E9476210E94F91C0E94F01B83E4A9
:1018D0000E94C51A8AE30E94C51A6BE080EB0E9441
:1018E00076219927182F00276AE080EB0E94762145
:1018F0009927082B192BC8010E94461C0E94F01B37
:1019000088E40E94C51A8AE30E94C51A68E080EB49
:101910000E9476210E94F91C0E94F01B8CE40E9418
:10192000C51A8AE30E94C51A69E080EB0E947621FD
:101930000E94F91C0E94F01B83E50E94C51A8AE3ED
:101940000E94C51A6CE080EB0E9476210E94F91C6F
:1019500045C00E94AB1842C00E94A2183FC00E941E
:10196000DE183CC080E494E00E94F91A0E94001C3A
:101970000E94471933C081E294E00E9452242EC095
:1019800088E897E00E94822329C081E00E94211A02
:1019900025C08AE30E94C51A0E94001C8093EE02B3
:1019A000109221016BE171E084E794E00E94DA2457
:1019B0008BE191E00E94D9230E94DF1781E08093A0
:1019C00021016BE171E084E794E00E94DA248BE16D
:1019D00091E00E94D92302C00E949520FF2011F4BB
:1019E0000C94AD0481E080930001FF24F09221016A
:1019F0006BE171E084E794E00E94DA248BE191E0EE
:101A00000E94D9230C948A04879903C081E00E9424
:101A1000211A869903C081E00E944C1A68E97AE392
:101A200087E392E00E94682468E97AE387E392E022
:101A30000E94682468E97AE387E392E00E946824C0
:101A40001092EE0261E088E00E94421761E080E0BF
:101A50000E94AE1762E080E00E94421760E086EAD2
:101A60009FEF0E94761781E00E941C1761E08EE2D2
:101A70000E94421781E00E941C1760E086EA9FEFF7
:101A80000E94761763E080E00E944217C1E0C09395
:101A9000EE028C2F0E948E178C1711F40E94DF1714
:101AA0008C2F0E941C1763E080E00E94421762E0C6
:101AB00080E00E94421760E086EA9FEF0E9476175E
:101AC0008C2F0E941C1762E080E00E94421780E089
:101AD0000E941C1760E08AE590E00E94761763E0A0
:101AE00080E00E94AE1712E01093EE028C2F0E944D
:101AF0008E17813011F40E94DF1763E08C2F0E9453
:101B0000AE17612F8C2F0E94AE1760E086EA9FEF20
:101B10000E9476178C2F0E941C176C2F83E30E9463
:101B200042176C2F80E00E94AE176C2F88E10E9454
:101B300042178C2F0E941C1760E086EA9FEF0E94DC
:101B400076176C2F81E30E944217612F80E00E947C
:101B5000AE1760E08AE590E00E94761780E00E9470
:101B60001C1763E080E00E94AE1703E00093EE02D2
:101B70008C2F0E948E17813011F40E94DF17602F86
:101B80008C2F0E94AE17612F8C2F0E94AE1760E041
:101B900086EA9FEF0E9476178C2F0E941C176C2FED
:101BA0008C2F0E94AE17612F80E00E94421760E0E8
:101BB00086EA9FEF0E9476178C2F0E941C176C2FCD
:101BC0008C2F0E94AE17612F80E00E94421780E0A8
:101BD0000E941C1760E08AE590E00E94761780E082
:101BE0000E941C176C2F80E30E94421780E00E9425
:101BF0001C1760E08AE590E00E947617602F80E075
:101C00000E94421784E08093EE0280E00E948E17CB
:101C1000813011F40E94DF1781E294E00E94522487
:101C200083E0809348018EE792E00E94E3248C01D8
:101C3000EE2481E080934A0180935101E092C60333
:101C4000F80184819581AA2797FDA095BA2FBC0140
:101C5000CD010E94E525DC01CB0128E93FEB42E103
:101C60005FE3BC01CD010E948225DC01CB01BC01F8
:101C7000CD010E94C825DC01CB01EC0197FD0BC012
:101C800082E290E090934D0180934C0190934F013C
:101C900080934E010DC08EED9FEF90934D01809388
:101CA0004C0190934F0180934E01D095C195DF4F29
:101CB00064E471E084E794E00E94DA2484E491E033
:101CC0000E94D9232097A1F5F1E0EF1609F43FC057
:101CD0000E94992086E00E94C319C82F87E00E94C5
:101CE000C319F82E80E00E94DF19803110F482E0E1
:101CF00017C0F80186818130B9F09091DF029C17FE
:101D000010F09F1588F49C1718F481E08093C603A7
:101D10009F1528F48091C6038E5F8093C60383E0ED
:101D2000F801878341E0E42EF1E0EF1689F60FC059
:101D300021978FEFCF3FD80739F00E949920219744
:101D4000EFEFCF3FDE07C9F781E0F80187831092FC
:101D50004D0110924C0110924F0110924E0164E41B
:101D600071E084E794E00E94DA2484E491E00E9428
:101D7000D92310924A0164E471E084E794E00E9460
:101D8000DA2484E491E00E94D923C8010E94F02360
:101D90004ACF85E08093560181E080935F0100E0A7
:101DA00080E00E94DF19182F81E00E94DF19C82F00
:101DB00083E00E94DF191F3020F0C33010F0833021
:101DC000D8F421E0209358018C1748F48CE090E07F
:101DD00090935D0180935C0184EF9FEF08C084EFD6
:101DE0009FEF90935D0180935C018CE090E0909375
:101DF0005B0180935A010BC020E0209358011092A0
:101E00005B0110925A0110925D0110925C01201743
:101E100059F0022F62E571E084E794E00E94DA2431
:101E200082E591E00E94D92360EF70E08FE296E0B6
:101E30000E946824B5CF82E08093640181E08093A2
:101E40006D0180936C0183E995E00E94E3248C018D
:101E500081E080936601F80110861092690110926A
:101E6000680110926B0110926A0160E671E084E7EC
:101E700094E00E94DA2480E691E00E94D9230E9437
:101E80007820F801868124813581813071F5809137
:101E90002E0290912F02E901C81BD90B1C161D06BA
:101EA0001CF421E030E002C02FEF3FEFCE01D7FF5E
:101EB00004C0882799278C1B9D0BE8E6F1E0BF0141
:101EC0000E94B127EC01853B910534F0E81BF90B2A
:101ED000EF01309521953F4FC29FC001C39F900DE8
:101EE000D29F900D1124EC0101C0E9011C161D06C2
:101EF0006CF480E09EE0909369018093680180E03B
:101F000092EF90936B0180936A010FC080E092EF93
:101F1000909369018093680180E09EE090936B014B
:101F200080936A01D095C195DF4F60E671E084E748
:101F300094E00E94DA2480E691E00E94D923219760
:101F40009FEFCF3FD907C9F00E949920F801F78091
:101F5000F1E0FF1669F40B9906C062E080EB0E9485
:101F60007621813029F4F801F0860E949E2005C078
:101F70002197FFEFCF3FDF0739F7109269011092E9
:101F8000680110926B0110926A0160E671E084E7CB
:101F900094E00E94DA2480E691E00E94D9230E9416
:101FA00078201092660160E671E084E794E00E9478
:101FB000DA2480E691E00E94D923C8010E94F02330
:101FC00042CF81E08093720180937B018DEC94E09D
:101FD0000E94E3248C01FC0194801092C603CC245F
:101FE000DD24AA2481E0809374010E949920992025
:101FF00031F481E00E94DF19F82E82E005C083E011
:102000000E94DF19F82E84E00E94DF19C82F80E0BB
:102010000E94DF19B82E80910201882389F00E9466
:10202000F01B8B2D0E94F91C8DE20E94C51A8F2D8A
:102030000E94F91C8DE20E94C51A8C2F0E94F91C87
:1020400086E00E94C319E82E87E00E94C319282F5A
:10205000FFE0FB1530F082E0F8018683F1E0AF2E5F
:102060008EC0F80185818130C1F09091DF029E150C
:1020700010F0921790F49E1518F481E08093C60337
:10208000921728F48091C6038E5F8093C603E1E027
:10209000AE2E83E0F801868372C0F8E1FF1508F4E4
:1020A00060C0FC1708F45DC0A6012C2F33278F2DCC
:1020B00099276901C81AD90ACC0CDD1C820F931F1D
:1020C00095958795C81AD90A68E070E0C60ED71EA4
:1020D0008091DA029927C89E9001C99E300DD89E42
:1020E000300D1124C601841B950BAC018091DB02DD
:1020F0009927489FF001499FF00D589FF00D11243A
:102100002E0F3F1FC9016AE070E00E94B127EB016A
:1021100080910201882331F08AE30E94C51ACE0122
:102120000E94B31C9E012E5D3F4F992069F43093AD
:1021300077012093760182E290E08C1B9D0B9093B7
:102140007901809378011BC082E290E08C1B9D0B8B
:1021500090937701809376013093790120937801F1
:102160000EC0F8E1FF1538F4FC1728F061E0A62E48
:10217000F801A68204C051E0A52EF8011682F1E014
:10218000AF1651F4109277011092760110927901F6
:1021900010927801109274016EE671E084E794E089
:1021A0000E94DA248EE691E00E94D92361E0A6160F
:1021B00031F062ED70E088E892E00E946824AA2085
:1021C00009F413CFC8010E94F02300CF89E0809367
:1021D000800181E0809389018DED94E00E94E324E9
:1021E0007C01FC01D48000E010E0E801CC2481E017
:1021F00080938201109385010093840110938701DD
:10220000009386018583F2E0DF1609F0C1C086E005
:102210000E94C319182F87E00E94C319082F9091BC
:10222000C603913011F0933079F48091DF02811769
:1022300058F082EF9FEF9093850180938401D093B3
:102240008701C093860110C09130C1F08091DF02F8
:102250008117A0F08EE090E0909385018093840137
:1022600010928701109286016CE771E084E794E098
:102270000E94DA248CE791E00E94D9230E949920E1
:1022800086E00E94C319182F8091DF028117B0F7F2
:10229000109285011092840110928701109286019C
:1022A0006CE771E084E794E00E94DA248CE791E027
:1022B0000E94D9239091C603892F8250823058F40E
:1022C0008091DF02801738F010928501109284010E
:1022D00082EF9FEF0CC09230C1F08091DF02801737
:1022E000A0F010928501109284018EE090E090930E
:1022F0008701809386016CE771E084E794E00E9497
:10230000DA248CE791E00E94D9230E94992087E08B
:102310000E94C319082F8091DF028017B0F7109236
:1023200085011092840110928701109286016CE75A
:1023300071E084E794E00E94DA248CE791E00E9447
:10234000D9230E94782088E090E090938F018093B9
:102350008E016AE871E08EE792E00E94DA248AE852
:1023600091E00E94D923109285011092840110926D
:10237000870110928601109282016CE771E084E778
:1023800094E00E94DA248CE791E00E94D92384C073
:102390000E949920DD2031F481E00E94DF19C82FCE
:1023A00082E005C083E00E94DF19C82F84E00E940C
:1023B000DF198C1729F4A1E0CA2EF701C5824AC0A3
:1023C000C93110F4893160F0C93118F083EF9FEF03
:1023D00002C08DE090E090938501809384012DC030
:1023E000A801082F11270C1B11098091DA029927E7
:1023F000089F9001099F300D189F300D1124B801DE
:10240000641B750B8091DB029927689FF001699F1F
:10241000F00D789FF00D11242E0F3F1FC9016AE0C7
:1024200070E00E94B12788279927861B970BDD2033
:1024300049F47093850160938401909387018093A0
:10244000860108C090938501809384017093870171
:1024500060938601F1E0CF1651F41092850110923D
:1024600084011092870110928601109282016CE71C
:1024700071E084E794E00E94DA248CE791E00E9406
:10248000D923CC2031F062ED70E081ED94E00E9420
:102490006824CC2009F47CCFC7010E94F0239CCE95
:1024A00084E08093960181E080939F01809398015E
:1024B000332484EE92E00E94E3245C01FC016480FA
:1024C0007580868097804084518480912A02909103
:1024D0002B02E301C81BD90B80912C0290912D0295
:1024E0006401C81AD90ACE01AA2797FDA095BA2F70
:1024F000BC01CD010E94E5257B018C01C601AA2704
:1025000097FDA095BA2FBC01CD010E94E525DC0105
:10251000CB01A8019701BC01CD010E944525DC013A
:10252000CB01B05820EE3EE245E652E4BC01CD01BD
:102530000E940127DC01CB01BC01CD010E94C8250E
:10254000DC01CB019093A5018093A40181E08093ED
:10255000A60160EA71E083E995E00E94DA2480EA4E
:1025600091E00E94D9230E94992080912A029091A3
:102570002B02E301C81BD90B80912C0290912D02F4
:102580006401C81AD90ACE01AA2797FDA095BA2FCF
:10259000BC01CD010E94E5257B018C01C601AA2763
:1025A00097FDA095BA2FBC01CD010E94E525DC0165
:1025B000CB01A8019701BC01CD010E944525DC019A
:1025C000CB01B05820EE3EE245E652E4BC01CD011D
:1025D0000E940127DC01CB01BC01CD010E94C8256E
:1025E000DC01CB019C012296259758F482E090E013
:1025F000C80ED91E95E0C916D10418F4B1E03B2EDF
:1026000054C080912E0290912F02281B390BC901D2
:10261000121613061CF4E1E0F0E002C0EFEFFFEF4A
:102620009C0197FF04C022273327281B390BC8E6DB
:10263000D1E0C901BE010E94B127853B910534F06C
:10264000C81BD90BCE01F095E195FF4F8E9F9001ED
:102650008F9F300D9E9F300D1124C901820F931F53
:102660006AE070E00E94B1279B012C5E3F4F3093DF
:102670009B0120939A012451304084E190E0821B19
:10268000930B90939D0180939C0162E971E084E734
:1026900094E00E94DA2482E991E00E94D92364EB5D
:1026A00070E086E395E00E94682431E0331609F07B
:1026B0005ACF10929B0110929A0110929D01109294
:1026C0009C0162E971E084E794E00E94DA2482E9E7
:1026D00091E00E94D9235092A5014092A40130922A
:1026E000A60160EA71E083E995E00E94DA2480EABD
:1026F00091E00E94D92310929B0110929A011092AE
:102700009D0110929C011092980162E971E084E7AA
:1027100094E00E94DA2482E991E00E94D923C50165
:102720000E94F023C5CE87E08093AD0181E08093C5
:10273000B60180E493E00E94E3247C0181E0809371
:10274000AF0162E080EB0E947621882309F58BE0DF
:1027500090E09093B2018093B10185EF9FEF909349
:10276000B4018093B30169EA71E084E794E00E94C8
:10277000DA2489EA91E00E94D92302C00E949920BC
:1027800062E080EB0E9476218823C1F30E949E20A4
:1027900064E080EB0E94762186E00E94C31987E006
:1027A0000E94C319CDE00E94992086E00E94C319BF
:1027B000182F87E00E94C3199091DF02911710F043
:1027C000981708F4C15062E080EB0E9476218823BC
:1027D00061F164E080EB0E947621282F80E490E094
:1027E000821B9109880F991F6AE070E00E94B1274F
:1027F000CB01162F0E949B1C8DE20E94C51A81E01E
:102800008093AF01212F332727FD309580E190E0A1
:10281000821B930B9093B2018093B101205F3F4FD5
:102820003093B4012093B3010AC080E190E090930B
:10283000B2018093B1019093B4018093B30169EA2E
:1028400071E084E794E00E94DA2489EA91E00E9432
:10285000D923CC2309F0A7CF0E949E201092B20169
:102860001092B1011092B4011092B30169EA71E0C3
:1028700084E794E00E94DA2489EA91E00E94D92357
:102880008C2F0E94211A64E080EB0E947621282F71
:1028900080E490E0821B9109880F991F6AE070E044
:1028A0000E94B127162F42C00E94992062E080EB5F
:1028B0000E947621882321F164E080EB0E9476213A
:1028C000282F80E490E0821B9109880F991F6AE00D
:1028D00070E00E94B127162F81E08093AF01262F70
:1028E000332727FD309588279927821B930B9093D8
:1028F000B2018093B1013093B4012093B3010CC0B5
:1029000085EF9FEF9093B2018093B1018BE090E04F
:102910009093B4018093B30169EA71E084E794E095
:102920000E94DA2489EA91E00E94D923812F992715
:1029300087FD909597FF03C0909581959F4F0297D3
:102940000CF0B2CF1092B2011092B1011092B4010A
:102950001092B30169EA71E084E794E00E94DA24FE
:1029600089EA91E00E94D9231A9A60EC7DE587E21A
:1029700094E00E9468241A9860E777E187E294E087
:102980000E946824C7E050C062E080EB0E9476217C
:102990008130F9F41092BD011092BE018C2F99275D
:1029A000909581959F4F9093BC018093BB0167EBFD
:1029B00071E083E995E00E94DA2487EB91E00E94C0
:1029C000D9231A9A60EC7DE587E294E00E9468249E
:1029D0001A9860E777E187E294E00E94682462E059
:1029E00080EB0E9476218130F1F41092BD011092AB
:1029F000BE018C2F9927880F991F9093BC0180935B
:102A0000BB0167EB71E083E995E00E94DA2487EB74
:102A100091E00E94D9231A9A60EC7DE587E294E068
:102A20000E9468241A98CF5F62E080EB0E947621B2
:102A3000813009F4A9CF81E0F70184831092B201BB
:102A40001092B1011092B4011092B3011092AF0133
:102A500069EA71E084E794E00E94DA2489EA91E06F
:102A60000E94D923C7010E94F02363CE85ED92E036
:102A70000E94E324EC011C8280E190E09093C50168
:102A80008093C40111E01093C60160EC71E08EE701
:102A900092E00E94DA2480EC91E00E94D9238D819B
:102AA000811719F41092D50102C01093D50161ED80
:102AB00071E08DED94E00E94DA2481ED91E00E94B6
:102AC000D9230E9495201092CE018D81813019F476
:102AD00084EB90E002C08CE49FEF9093CD01809353
:102AE000CC0181E08093CF0168EC71E083E995E04F
:102AF0000E94DA2488EC91E00E94D9231091D00141
:102B0000113021F481E20E94C51A1C83CE010E947B
:102B1000F023ACCF86E08093DD0181E08093E60175
:102B20001092DF011092DE0186E190E09093E201C5
:102B30008093E1019093E4018093E30169ED71E0FA
:102B400084E794E00E94DA2484E794E00E94E3247E
:102B50009093D8018093D70180910101882369F077
:102B600088E20E94C51AE091D701F091D8018481D2
:102B70000E94F91C8EE30E94C51AA091D701B09162
:102B8000D80114968C9114978B3020F0CD010E94BF
:102B9000F023DACF9927FC0153E0EE0FFF1F5A957F
:102BA000E1F7E80FF91FE953FC4F16968C91169741
:102BB000818314968C9114979927FC0143E0EE0FC2
:102BC000FF1F4A95E1F7E80FF91FE953FC4F1896EC
:102BD0008D919C9119978383948314968C9114976B
:102BE0009927FC0133E0EE0FFF1F3A95E1F7E80F5C
:102BF000F91FE953FC4F1A968D919C911B97858381
:102C0000968314968C9114979927FC0123E0EE0F7C
:102C1000FF1F2A95E1F7E80FF91FE953FC4F1D96B6
:102C20008C911D97808714968C9114979927FC019D
:102C300003E0EE0FFF1F0A95E1F7E80FF91FE953D4
:102C4000FC4F1C968C911C978783CD010E94F0232A
:102C500020E0022FC0E0222371F58C2F9927FC0180
:102C600013E0EE0FFF1F1A95E1F7E80FF91FE95384
:102C7000FC4F80818130D1F482818017B9F41181B9
:102C80001130A1F489E0C89FC001112489539C4FE1
:102C90000E942F2080910101882339F08C2F805DC4
:102CA0000E94C51A89E20E94C51A212FCF5FCA303F
:102CB00010F4222391F20F5F093010F4222351F215
:102CC000222379F480910101882319F08DE20E947A
:102CD000C51A1092A9061092A80610924B061092DF
:102CE0004A06C79B02C0C7982FCFC79A2DCF90E046
:102CF000E7ECF3E0118210821382148215821682AF
:102D000081E080871782980F39969A3098F38093E4
:102D1000C7038093D0038093EB038093D903809300
:102D2000E2038093060480930F0480931804809339
:102D3000F4038093C90382E08093F60383E08093D9
:102D4000D20396E09093ED0384E08093DB038093BD
:102D5000E40388E08093FF039093080490931104A8
:102D600090931A040895CFEFD0E1DEBFCDBF80E08D
:102D700090E00E94762330E235BF86EF82BF96E076
:102D800093BF21E027BF8FEF8ABB1BBA87BB18BA5E
:102D900084BB15BA8CE381BB12BA92B913B83093D5
:102DA00061001092620081EA8FBD2EBD8FE788BD61
:102DB0008ABD0E94B81983E390E00E94B11A8BE2A9
:102DC0008CB98CB90E94F2200E94A2180E9477163A
:102DD0000E94031A84EA98E00E94822389E497E023
:102DE0000E94822380E597E00E94822388E897E092
:102DF0000E94822387E597E00E9482238CE697E079
:102E00000E9482238EE597E00E94822385E697E068
:102E10000E94822381E897E00E9482238AE797E05C
:102E20000E9482238FE897E00E9482230E943D2324
:102E300080E090E00C94FB278093EB0167EE71E05B
:102E40008DED94E00E94DA2487EE91E00E94D92370
:102E50008091EC01813091F085EC92E00E94F91AAA
:102E600081E40E94C51A8091EC010E94F91C8FE751
:102E700088BD8ABD81E294E00E9452248091EC01D9
:102E800099270895CF93C62F99279093F2018093A5
:102E9000F101633019F41092F30103C081E08093D3
:102EA000F3016DEE71E08EE792E00E94DA248DEE80
:102EB00091E00E94D9238091F4018C1791F085EC68
:102EC00092E00E94F91A86E40E94C51A8091F401EA
:102ED0000E94F91C8FE788BD8ABD81E294E00E94C0
:102EE00052248091F4019927CF9108950F931F9355
:102EF00009EF11E09093FA018093F9016093FC01CE
:102F0000B8016450704083E995E00E94DA24C8015A
:102F100004970E94D9231F910F9108958093030273
:102F20006EEF71E085ED92E00E94DA248EEF91E081
:102F30000E94D92380910202813069F464E072E03A
:102F400080E493E00E94DA2484E092E00E94D92396
:102F500081E090E0089580E090E00895CF93C62F3F
:102F600080930D02633019F410920E0203C081E0C9
:102F700080930E0269E072E08DEC94E00E94DA2406
:102F800089E092E00E94D92380910F028C1791F082
:102F900085EC92E00E94F91A84E50E94C51A80919E
:102FA0000F020E94F91C8FE788BD8ABD81E294E080
:102FB0000E94522480910F029927CF910895CF93B8
:102FC000109215021092140210921702109216021B
:102FD00084EB90E0909319028093180260E172E014
:102FE00084EE92E00E94DA2480E192E00E94D923EC
:102FF000C091EE028C2F81508230E0F5C130A1F4F7
:103000008C2F0E941C1763E080E00E94421762E050
:1030100080E00E94421760E08AE590E00E94761707
:1030200080E00E941C1716C0C230A1F463E081E06A
:103030000E94AE176C2F81E00E94AE1760E086EA16
:103040009FEF0E94761781E00E941C1761E08FE2DB
:103050000E94421761E080E30E94421760E08AE527
:1030600090E00E94761761E083E30E94421763E0DC
:1030700081E057C08C2F8350823008F055C0C33098
:10308000A1F56C2F81E00E94AE1762E081E00E9402
:10309000AE1760E086EA9FEF0E94761781E00E94FB
:1030A0001C1761E0862F0E94AE1762E080E00E944C
:1030B000421760E086EA9FEF0E94761781E00E9447
:1030C0001C1761E0862F0E94AE1762E080E00E942C
:1030D000421780E00E941C1760E08AE590E00E94A1
:1030E000761780E00E941C170EC0C43081F480E087
:1030F0000E941C1762E080E00E94421760E08AE5AF
:1031000090E00E94761762E080E00E94AE1780E0B7
:103110000E941C1760E08AE590E00E94761763E049
:1031200080E00E94AE170AC085EC92E00E94F91A76
:1031300086E997E00E94F91A0E9445240E944524DE
:10314000CF9108954BE050E060E070E089ED92E0AF
:103150000E94CD22089564E181E090E00E94DE2289
:103160006AE082E090E00E94DE226BE183E090E082
:103170000E94DE2260E084E090E00E94DE2261E2B4
:1031800085E090E00E94DE226FE886E090E00E94F9
:10319000DE2266E087E090E00E94DE2260E088E0C8
:1031A00090E00E94DE2266EE89E090E00E94DE223E
:1031B00064E08AE090E00E94DE22089589EF92E0C8
:1031C0000E94F91A88E293E00E94F91A81E090E0E7
:1031D0000E94C5220E94F91C85E493E00E94F91A1E
:1031E00082E090E00E94C5220E94F91C82E693E0F2
:1031F0000E94F91A83E090E00E94C5220E94F91C07
:103200008EE793E00E94F91A84E090E00E94C522C4
:103210000E94F91C8AE993E00E94F91A85E090E087
:103220000E94C5220E94F91C86EB93E00E94F91AC5
:1032300086E090E00E94C5220E94F91C84ED93E094
:103240000E94F91A87E090E00E94C5220E94F91CB2
:103250008EEE93E00E94F91A88E090E00E94C52269
:103260000E94F91C87E094E00E94F91A89E090E03E
:103270000E94C5220E94F91C8EE194E00E94F91A76
:103280008AE090E00E94C5220E94F91C08951F93D5
:10329000182F8DE30E94C51A812F9927853091053B
:1032A00009F43FC08630910594F48230910539F1DC
:1032B0008330910534F4009709F458C00197C9F0A0
:1032C00055C08330910509F1049729F14FC088302A
:1032D0009105C9F18930910534F48630910539F1B1
:1032E000079759F143C08930910599F10A97B9F1CF
:1032F0003DC00E94001C682F81E090E035C00E9414
:10330000001C682F82E090E02FC00E94001C682FF4
:1033100083E090E029C00E94001C682F84E090E0C8
:1033200023C00E94001C682F85E090E01DC00E9411
:10333000001C682F86E090E017C00E94001C682FD8
:1033400087E090E011C00E94001C682F88E090E0A8
:103350000BC00E94001C682F89E090E005C00E940D
:10336000001C682F8AE090E00E94DE221F910895E1
:103370008AE192E00E94F22385E886B980E287B96B
:1033800080E180BD08951F93182F8AE192E00E948A
:10339000DB239FB7F89487B1807E87B91F7187B10F
:1033A000812B87B9349A369A349BFECF9FBF8AE12E
:1033B00092E00E94F22385B199271F9108950F93FF
:1033C0001F93CF93DF93082FC0E0D0E010E0802F51
:1033D0000E94C319E82FFF27EB55F84F8491C80FBF
:1033E000D11D1F5F123098F3D695C7958C2FCF3F14
:1033F00019F48FEF90E002C08A509927DF91CF91A6
:103400001F910F9108954091E10264E180EB0E94C9
:10341000CC214091E00265E180EB0E94CC214091FB
:10342000E3026CE080EB0E94CC214091E20267E075
:1034300080EB0E94CC2141E0642F80EB0E94CC21E4
:103440000895CF93C82FC09A41E06DE080EB0E94B1
:10345000CC216DE080EB0E9476218823D1F7C098C3
:1034600062E080EB0E9476218130A1F4C13091F4BA
:1034700065E180EB0E947621682F87E090E00E9452
:10348000DE2264E180EB0E947621682F88E090E0E4
:103490000E94DE22CF910895AF92BF92CF92DF9229
:1034A000EF92FF920F931F93CF93DF93A82EEE24FA
:1034B000FF246701BB2486E00E94C3199927C81620
:1034C000D90630F486E00E94C319082F112701C0E5
:1034D0008601680187E00E94C3199927E816F9065A
:1034E00030F487E00E94C319C82FDD2701C0E7012F
:1034F0007E01B39483E08B15F0F6C8010E94461C50
:103500008DE20E94C51ACE010E94461CC8010C170C
:103510001D0708F4CE018093DF028DE30E94C51AD7
:103520008091DF0299270E94461C8DE30E94C51AF4
:103530008091DF0299270E94461C81E0A81631F491
:103540006091DF0286E090E00E94DE22DF91CF9161
:103550001F910F91FF90EF90DF90CF90BF90AF90B1
:1035600008950F931F938C018AE396E00E94F22343
:10357000812F99278093900009B988E98AB986E05C
:10358000809395001F910F910895CF93C82F8AE3E0
:1035900096E00E94DB235D9905C0559A86E396E08C
:1035A0000E94DB23CCB98AE396E00E94F22380E0FC
:1035B00090E0CF91089588E396E00E94DB2380910C
:1035C00035069927089555980E94F12286E396E0E2
:1035D0000E94FC230E943D2357980E94F1228CB147
:1035E0008093350688E396E00E94FC23579A0E9458
:1035F0003D23CF93DF93EC01FC0121968491882336
:1036000039F00E94C51AFE01219684918823C9F7DA
:10361000DF91CF9108951F930E94DB1A182F0E940B
:10362000C51A812F99271F91089584E00E94231BBA
:10363000089582E00E94231B9927089581E00E944B
:10364000231B99270895AF92BF92DF92EF92FF92CA
:103650000F931F93CF93DF93CDB7DEB721970FB6AC
:10366000F894DEBF0FBECDBFAA24BB24D82E88237A
:1036700089F10E94DB1A182F898399270E94E2277B
:10368000892BB9F3812F0E94C51A8981E82EFF2466
:10369000C7010E94DA270D2D1127DA94892B39F002
:1036A000C7010E94EB2789838753992704C0CE0165
:1036B00001960E949922000F111F000F111F045044
:1036C000104002C0880F991F0A95E2F7A80EB91E94
:1036D000DD2079F6C50121960FB6F894DEBF0FBE46
:1036E000CDBFDF91CF911F910F91FF90EF90DF90B1
:1036F000BF90AF900895EF92FF920F931F937B01BD
:103700008C0180E30E94C51A88E70E94C51AC8018F
:10371000AA27BB2762E00E94C41B62E0C7010E9487
:10372000C41B1F910F91FF90EF9008950F931F936B
:103730008C0180E30E94C51A88E70E94C51A62E0E6
:10374000C8010E94C41B1F910F9108951F93182F49
:1037500080E30E94C51A88E70E94C51A812F992725
:1037600061E00E94C41B1F9108951F93182F80E3EE
:103770000E94C51A88E70E94C51A812F0E94F71B74
:103780000E94C51A1F9108950F931F93CF93DF9343
:103790008C01623080F0C12FDD27C801892F992765
:1037A00082958F700E94F71B0E94C51A8C2F0E9471
:1037B000F71B0E94C51AE80144E0D695C7954A95C3
:1037C000E1F78C2F0E94F71B0E94C51A802F0E94E0
:1037D000F71B0E94C51ADF91CF911F910F91089599
:1037E0008DE00E94C51A8AE00E94C51A08958F7064
:1037F0008A3010F0895C01C0805D99270895089592
:103800000F931F93CF930E94DB1AC82F80538A30E7
:1038100030F00E94DB1AC82F80538A30D0F78C2FEB
:103820000E94C51A84E6C89F80011124005C1241E1
:103830000E94DB1AC82F80538A3030F00E94DB1AB6
:10384000C82F80538A30D0F78C2F0E94C51A8AE087
:10385000C89FC0011124080F191F005E11400E946B
:10386000DB1AC82F80538A3030F00E94DB1AC82F31
:1038700080538A30D0F78C2F0E94C51AC8018C0F54
:10388000911DC097CF911F910F910895CF93DF9312
:10389000EC0180E0209711F480E348C097E2C0314A
:1038A000D90738F0C051D7428F5F97E2C031D907AE
:1038B000C8F7882311F4209719F4805D0E94C51A77
:1038C00080E093E0C83ED90738F0C85ED3408F5FF0
:1038D00093E0C83ED907C8F7882311F4209719F45C
:1038E000805D0E94C51A80E0C436D10530F0C45610
:1038F000D0408F5FC436D105D0F7882311F42097CC
:1039000019F4805D0E94C51A80E0CA30D10528F004
:103910002A978F5FCA30D105D8F7882311F42097F2
:1039200019F4805D0E94C51A8C2F805D0E94C51A13
:10393000DF91CF910895CF93C82F181614F48BE21E
:1039400003C087FF03C08DE20E94C51A8C2F992700
:1039500087FD909597FF03C0909581959F4F0E949A
:10396000F91CCF910895CF93DF93EC011816190637
:1039700014F48BE203C097FF03C08DE20E94C51AC6
:10398000CE01D7FF03C0909581959F4F0E94461CA2
:10399000DF91CF91089518161CF087FF03C0819521
:1039A0009927089580E090E0089508951816190663
:1039B00044F097FF04C0909581959F4F089580E053
:1039C00090E0089508950F931F93CF93082F10E868
:1039D000C0E0802F812311F081E301C080E30E94C9
:1039E000C51A1695CF5FC830A0F3CF911F910F91E4
:1039F0000895CF93C82F80E0CC2311F480E31DC03D
:103A0000C43620F0C4568F5FC436E0F7882311F423
:103A1000CC2319F4805D0E94C51A80E0CA3020F0E2
:103A2000CA508F5FCA30E0F7882311F4CC2319F411
:103A3000805D0E94C51AC05D8C2F0E94C51ACF916F
:103A40000895FF920F931F93CF930E94DB1AC82F04
:103A50008D3211F4FF2403C071E0F72E8BE20E9437
:103A6000C51A8C2F80538A3030F00E94DB1AC82F81
:103A700080538A30D0F78C2F0E94C51A84E6C89FE5
:103A800080011124005C12410E94DB1AC82F805370
:103A90008A3030F00E94DB1AC82F80538A30D0F76A
:103AA0008C2F0E94C51A8AE0C89FC0011124080FFC
:103AB000191F005E11400E94DB1AC82F80538A3004
:103AC00030F00E94DB1AC82F80538A30D0F78C2F39
:103AD0000E94C51A0C0F111D00531040FF2029F43D
:103AE00088279927801B910B01C0C801CF911F9196
:103AF0000F91FF9008950E94291F68E770E081E30D
:103B000092E00E946A248EEA96E00E94F223F894E2
:103B100000911D0210921D02E0901C0210921C02E6
:103B20007894602F8EE996E00E9460206E2D80E4EC
:103B300096E00E9460208091AD068130F1F41092F1
:103B4000AD0680E090E0A0E0B0E080931E0290938C
:103B50001F02A0932002B09321028093220290932F
:103B60002302A0932402B09325028093260290930F
:103B70002702A0932802B0932902112707FD109570
:103B8000FF24E7FCF094C8018E199F09AA2797FD2E
:103B9000A095BA2FBC01CD010E94E525DC01CB0127
:103BA0002EE231E04EEA59E3BC01CD010E9401272B
:103BB0003B014C010E0D1F1DC801AA2797FDA095C2
:103BC000BA2FBC01CD010E94E525DC01CB012CEB15
:103BD0003DE14AE05CE3BC01CD010E9401275B01AD
:103BE0006C018091260290912702A0912802B09149
:103BF0002902A4019301BC01CD010E940325DC012F
:103C0000CB018093260290932702A0932802B093C1
:103C100029028091260290912702A0912802B0915A
:103C20002902BC01CD010E947425DC01CB019C015D
:103C3000AD01C601B5010E940127DC01CB01E09076
:103C40001E02F0901F0200912002109121029C019F
:103C5000AD01C801B7010E940325DC01CB018093AF
:103C60001E0290931F02A0932002B0932102809124
:103C7000260290912702A0912802B0912902BC014E
:103C8000CD010E944F27DC01CB019C01AD01C60193
:103C9000B5010E940127DC01CB01E0902202F090E7
:103CA000230200912402109125029C01AD01C8015C
:103CB000B7010E940225DC01CB0180932202909380
:103CC0002302A0932402B0932502809126029091B2
:103CD0002702A0912802B0912902A4019301BC01FE
:103CE000CD010E940325DC01CB0180932602909335
:103CF0002702A0932802B093290280912602909176
:103D00002702A0912802B09129022BED3FE049EC57
:103D100050E4BC01CD010E94052688238CF08091DF
:103D2000260290912702A0912802B09129022BED42
:103D30003FE049EC50E4BC01CD010E94022522C0C5
:103D40008091260290912702A0912802B091290229
:103D500020E030E040E050E0BC01CD010E940226AE
:103D60008823D4F48091260290912702A091280202
:103D7000B09129022BED3FE049EC50E4BC01CD01AC
:103D80000E940325DC01CB01809326029093270239
:103D9000A0932802B0932902F89480912602909172
:103DA0002702A0912802B091290220EE3EE245E6CA
:103DB00052E4BC01CD010E940127DC01CB01BC0112
:103DC000CD010E94C825DC01CB0190932F02809386
:103DD0002E0280911E0290911F02A0912002B091AC
:103DE0002102BC01CD010E94C825DC01CB019093CA
:103DF0002B0280932A028091220290912302A091AB
:103E00002402B0912502BC01CD010E94C825DC012D
:103E1000CB0190932D0280932C0278948AE996E04E
:103E20000E94871F8AE996E00E94CF1F8CE396E0EC
:103E30000E94871F8CE396E00E94CF1F80914E0660
:103E40008ABD8091AC0688BD81E392E00E94D923AF
:103E500054CE80E091E090934D0680934C06809183
:103E60004C0690914D069093AB068093AA06109253
:103E70004906109248068091480690914906909311
:103E8000A7068093A60610924B0610924A068091D0
:103E90004A0690914B069093A9068093A80610922B
:103EA00045061092440680914406909145069093F1
:103EB000A3068093A20610924706109246068091B0
:103EC0004606909147069093A5068093A40610920B
:103ED00040061092410610924206109243068091CD
:103EE000400690914106A0914206B091430680930E
:103EF0009E0690939F06A093A006B093A10681E032
:103F00008093AD0681B1807F809330020895FC01DB
:103F100024853585868597852817390784F4848517
:103F2000958520893189820F931F84879587248501
:103F300035858685978582179307A4F40FC08485FD
:103F4000958520893189821B930B848795872485E9
:103F50003585868597852817390724F486859785C2
:103F60008487958764857585CF010E94B81F089561
:103F7000FC01CB016FB7F8949C01442737FD4095B5
:103F8000542F80819181A281B381820F931FA41F3E
:103F9000B51F80839183A283B3836FBF0895CF93AE
:103FA000DF93FC0180819181A281B381292F3A2F77
:103FB0004B2F552747FD5A9584819581A681B7815E
:103FC000E901C81BD90B8091DC0299278C9FA001C5
:103FD0008D9F500D9C9F500D11248091DE02282F43
:103FE000332780859185BE01681B790BCB01289F03
:103FF000B001299F700D389F700D1124460F571F77
:104000008091DD02282F332782859385289FB00178
:10401000299F700D389F700D1124460F571FCA013C
:104020006AE070E00E94B127C087D1876F377105C1
:104030001CF06FE770E00DC08FEF623878071CF45A
:1040400061E87FEF06C0828593858C0F9D1F828774
:104050009387862F8058828BDF91CF910895CF93DD
:10406000DF93EC0188852B813C818130B1F4A9017B
:104070008F81813011F0522F44275093A90640932D
:10408000A8062D813E818F81813011F0322F2227A9
:1040900030934B0620934A0610C0922F8827BC010C
:1040A0008AE996E00E94B81F8D819E81982F88270B
:1040B000BC018CE396E00E94B81FDF91CF91089578
:1040C000FC01862F6FB7F894282F332727FD3095F2
:1040D000432F532F80819181A281B381820F931F3F
:1040E000A41FB51F80839183A283B3836FBF0895FC
:1040F0008091A6069091A706892B31F480914806FD
:1041000090914906892B81F08EEA96E00E94DB238C
:104110008091A6069091A706892BB1F78091480659
:1041200090914906892B81F7089581E08093AD062F
:1041300008958EEA96E00E94DB23089510924906C6
:104140001092480680914806909149069093A706E0
:104150008093A60610924B0610924A0680914A065A
:1041600090914B069093A9068093A806089541B1BB
:10417000407F30913002542F5327952F9695957597
:10418000852F880F8A7A982B592B242F2695232741
:104190002575842F9927880F991F38273A7A232B62
:1041A000522340933002252F332724FF05C08091EE
:1041B0001D028F5F80931D0225FF05C080911D02A7
:1041C000815080931D0226FF05C080911C028F5FE5
:1041D00080931C0257FF05C080911C028150809380
:1041E0001C0208958AEB96E00E94F22388E48093F3
:1041F00070001092710084E0809374000895282F5D
:1042000084EA809374008091740087FFFCCF8091D2
:1042100071009927887F9070089781F4209373002C
:1042200084E8809374008091740087FFFCCF8091B4
:1042300071009927887F9070489719F081E090E08D
:10424000089580E090E008950895282F84EA8093EF
:1042500074008091740087FFFCCF809171009927D2
:10426000887F9070409789F42093730084E880934E
:1042700074008091740087FFFCCF809171009927B2
:10428000887F90708034910519F081E090E0089566
:1042900080E090E00895089584E980937400089583
:1042A0008093730084E8809374008091740087FF8A
:1042B000FCCF809171009927887F9070889719F0C2
:1042C00081E090E0089580E090E0089508958130C5
:1042D00011F484EC01C084E8809374008091740030
:1042E00087FFFCCF80917300992708950F931F9348
:1042F000CF93C82F162F00E08AEB96E00E94DB23B5
:104300008C2F0E94FF20882371F08091B806909135
:10431000B90601969093B9068093B80682E70E9489
:10432000C51A81E326C0812F0E945021882371F095
:104330008091B8069091B90601969093B906809342
:10434000B80682E70E94C51A82E313C0CF5F8C2FA4
:104350000E942521882381F08091B8069091B906AA
:1043600001969093B9068093B80682E70E94C51A19
:1043700083E30E94C51A04C0802F0E946721082F82
:104380000E944C218AEB96E00E94F223802F99270D
:10439000CF911F910F910895FF920F931F93CF9389
:1043A000182FC62F042FFF248AEB96E00E94DB23F0
:1043B000812F0E94FF20882371F08091B806909190
:1043C000B90601969093B9068093B80687E70E94D4
:1043D000C51A81E326C08C2F0E945021882371F0DA
:1043E0008091B8069091B90601969093B906809392
:1043F000B80687E70E94C51A82E313C0802F0E9487
:104400005021F82E882379F08091B8069091B90652
:1044100001969093B9068093B80687E70E94C51A63
:1044200083E30E94C51A0E944C218AEB96E00E9409
:10443000F2238F2D9927CF911F910F91FF9008950F
:10444000FF920F931F93CF93C82FF62E00E010E03A
:104450008AEB96E00E94DB238C2F0E94FF208823AA
:1044600061F48F2D0E945021882339F4CF5F8C2F67
:104470000E942521C82F882351F08091B806909181
:10448000B90601969093B9068093B8060BC081E0F7
:104490000E9467219927182F00278C2F0E946721DF
:1044A000080F111D0E944C218AEB96E00E94F22316
:1044B000C801CF911F910F91FF900895FF920F9324
:1044C0001F93CF93DF93182F062FEA01FF248AEB67
:1044D00096E00E94DB23812F0E94FF20882391F425
:1044E000802F0E945021882369F48D2F99270E94E4
:1044F0005021F82E882331F48C2F0E945021F82E61
:10450000882349F08091B8069091B906019690935E
:10451000B9068093B8060E944C218AEB96E00E946F
:10452000F2238F2D9927DF91CF911F910F91FF904B
:104530000895FC0188279927E89421912223E9F026
:104540002032D9F32930C9F32A30B9F32C30A9F33A
:104550002D3099F3263789F32B3219F02D3221F4BF
:1045600068942191222349F020333CF02A332CF423
:1045700020532FD0820F911DF4CF8115910521F08A
:104580001EF48095909501960895E199FECF9FBB0A
:104590008EBBE09A99278DB308954115510569F0B6
:1045A000DC01E199FECF7FBB6EBBE09A6F5F7F4F6E
:1045B0000DB20D9241505040B1F70895E199FECFF0
:1045C0009FBB8EBB6DBB0FB6F894E29AE19A0FBE0B
:1045D00008957AE0979F902D879F802D910D11244B
:1045E0000895DF93CF93BF93AF939F93D6E0CCEB27
:1045F0009FB7AE81AF5FAE8360F0AA81BB81BA2B5B
:1046000041F4CDB7DEB7FE81EF812996CDBFDEBF85
:1046100009948F937F936F935F934F933F932F935F
:104620001F930F93FF92EF92DF92CF92BF92AF92C0
:104630009F928F927F926F925F924F923F922F92B2
:104640001F920F929F93CDB7DEB79B8D39A148A1E2
:10465000E8A3F9A370F0F6E0ECEBD381C281BEB71A
:10466000ADB7BD83AC8324812DBF25812EBFCA2F5A
:10467000DB2F1124E32FF42F0994EF91EF91ECEB52
:10468000F6E0F89406810A95068354F4D181C0813E
:10469000D383C283209639F1BD81AC81ADBFBEBF4B
:1046A0000F900FBE0F901F902F903F904F905F90F4
:1046B0006F907F908F909F90AF90BF90CF90DF9042
:1046C000EF90FF900F911F912F913F914F915F912C
:1046D0006F917F918F919F91AF91BF91CF91DF911A
:1046E000EF91FF91189578948895FDCFFF91EF9108
:1046F0008050904011F48DB79EB78093C006909380
:10470000C106099401D023C0E82FF92F1DD0A02D98
:104710001BD0B02D19D00C9217D00E9240E040E083
:1047200051E24E935A95E9F711970ED0802D0CD097
:10473000902D0AD0E82FF92FA483B5830382A0E639
:10474000A283418340830895C89531960895F894D3
:1047500048DF7894E82FF92F22812F7D228326FFCE
:1047600003C02F7B228301D08ACFE82FF92F3FEFA0
:1047700022812073D1F4CF932D2F4381CCEBD6E04F
:10478000F8943395EC2FFD2FC081D181209619F03C
:104790005B814517B0F791838083F92FE82FD18390
:1047A000C083CF91D22F832F1895832F206422832B
:1047B00018958E5F9F4FE82FF92FF8942081318153
:1047C0002150304019F42083318318950ADFECEB37
:1047D000F6E07381628137D0E82FF92F26D04FCFD2
:1047E0008E5F9F4F09D0882309F00895F894F9DE71
:1047F000789445CF8E5F9F4FE82FF92F81E090E0AE
:10480000F894718160818617970720F080839183E7
:104810008FEF18958FE586179707D0F723D07894F8
:10482000862F972FA2CFE22FF32F208131812050A6
:104830003040C9F771836083F72FE62F31832083DF
:104840000895F32FE22F208131816217730751F011
:1048500020503040B1F70895608171816050704000
:1048600009F408954C2F5D2FC62FD72F79816881C9
:1048700071836083E62FF72F6627688369837D2F16
:104880006C2FC42FD52F98940895F894FECFF894E8
:10489000A8DE7894F091BF06E091BE06228125FD46
:1048A00009C0EDCEF8949DDE7894F92FE82F22818F
:1048B000206222837F2F6E2FF6E0ECEBF894C3DFAB
:1048C000C22FD32F209619F0EA81E064EA83D7CE75
:1048D00001D06FCF6050704009F482CFF89481DE30
:1048E00078947FD0E4ECF6E0F8942091C6062A95FF
:1048F0002093C6067894CE2FDF2FE881F981309679
:1049000059F024813581621B730BA8F7620F731F66
:10491000261B370B2483358399838883D92FC82F8F
:10492000F983E8836C837D833CD0A9CEF8942091F1
:10493000C60621502093C606789408F00895CF93B8
:10494000DF93AF93BF93D091C506C091C406209664
:1049500021F1FD81EC813197FD83EC83EF2BE9F4AC
:10496000A881B981B093C506A093C406F983E883F2
:104970008A819B818250904031F48E819F817D2F6E
:104980006C2F1DD003C08C2F9D2F34DF109629F083
:10499000CA2FDB2FFD81EC81E1CFBF91AF91DF9179
:1049A000CF91F8942091C60623952093C60678945B
:1049B00031F60895F89415DE789401D060CEF92F81
:1049C000E82F33DF17CFE82FF92FF89445DF7894DD
:1049D00021F4EFDE82509040F6CF03D0862F972F40
:1049E0000895E82FF92F329602C0F92FE82FF89496
:1049F000408151814150504011F04F5F5F4F5183D2
:104A0000408318955058192EA9D101D040C1BA172A
:104A10006207730784079507B1F188F40EF41094C8
:104A20000B2EBA2FA02D062E622F202D072E732FAE
:104A3000302D082E842F402D092E952F502DFF2725
:104A40005523B9F0591B49F0573E98F046953795D4
:104A50002795A795F0405395C9F776F0BA0F621FD6
:104A6000731F841F30F4879577956795B795F0404D
:104A7000939517FA0F2E0895BF1BBB27BA0B620B35
:104A8000730B840BF6CFDEF685C1552319F09923FD
:104A900051F017C09923A1F097FB6BED7FE089ECF3
:104AA0009FE397F90895552359F02AF46BED7FE0C1
:104AB00089E490E408956627772788279927089541
:104AC000FEC01F93112797FD116057FD12601AD089
:104AD000F9D111FF07C02BED3FE049E450E410FD90
:104AE000506891DF1F91089550E449EC3FE02BEDB1
:104AF00076D0AAC0592F482F372F262F9FE380E862
:104B0000772766272BD101D0C2C0552359F09923AE
:104B100069F09F575F57951B33F442F4903811F4B6
:104B2000915805C0CCC091589F3F09F433C1BB27B1
:104B3000112462177307840730F4660F771F881FEC
:104B4000BB1F915098F311D00F920FD00F920DD040
:104B5000A0E82617370748071B0609F0A048BA2F18
:104B6000602D7F918F9100240895A0E800246217A2
:104B700073078407B10528F0621B730B840BB1091E
:104B80000A2A660F771F881FBB1FA69581F7089515
:104B900097FBF0D09F3738F0FEE9F91B982F872F4D
:104BA000762F6B2F05C0F3C09695879577956795FF
:104BB000F150D0F73EF490958095709561957F4FB8
:104BC0008F4F9F4F0895E89403C097FB0EF4F3DFD7
:104BD000B62F672F782F892F9EE9002458C05F7762
:104BE000552319F444230AF06AC02F933F934F933F
:104BF0005F9388DF55274427CFD05F914F913F9136
:104C00002F91FFC00ED05EF004C00BD026F001C083
:104C100008D019F020F48FEF089580E0089581E026
:104C2000089597FB092E052600F868949AD0E89419
:104C300007FC07C0621773078407950721F008F483
:104C400000940794989408951F939F7750EC49E43B
:104C50003FE02BEDD8DE10E89F775FE349EC3FE0C3
:104C60002BED621773078407950720F050EC49E499
:104C7000CADE1127C2D09068ECE3F1E023D091277F
:104C80001F9108959A95BB0F661F771F881F1124E7
:104C90009923A1F08823B2F79F3F59F0BB0F48F446
:104CA00021F4002011F460FF04C06F5F7F4F8F4F2D
:104CB0009F4F881F9795879597F9089568C09FEF34
:104CC00080EC0895092E56D0FF92EF92DF92CF929A
:104CD000BF92AF92B02CC92ED82EE72EF62EA590FB
:104CE00018D0A590AA2071F09F938F937F936F9314
:104CF0006F2D7E2D8D2D9C2D0CD02F913F914F919E
:104D00005F9103DFAF90BF90CF90DF90EF90FF9067
:104D1000BECF16D147FB406804C02F2D3E2D4D2D30
:104D20005C2DEF93FF9370D0FF91EF9109D1AA27EB
:104D300007F80B24102C042607FA4068FF9367DE5F
:104D4000FF91992341F0882332F09A95BB0F661F9B
:104D5000771F881FF8CFAA9401F70895052E09261A
:104D600007FA440F551F5F3F79F0AA27A51708F0EF
:104D700051E04795880F991F9F3F31F0BB27B91726
:104D800008F091E0879508959F919F9198CF6627AD
:104D9000772788279927089597FBECDFCF93DF9338
:104DA000D52FC42F55274427332722279923D9F0FD
:104DB0009F37C8F0F92F6BDF592F482F372F262F39
:104DC000F63968F4E5DE01DFC030CD0721F06993E4
:104DD0007993899399939058DF91CF9114CE992725
:104DE000882777276627C030CD0721F0299339938C
:104DF00049935993DF91CF914ACF592F482F372F9D
:104E0000262FACDF01D043CF992339F0552329F069
:104E10009F575F57950F13F4CAF1BCCF91589F3F2E
:104E2000E1F3A62F00241124BB2766275527F8E0BD
:104E3000A69520F4020E131EB41F651F220F331F08
:104E4000441F551FFA95A1F7F8E0E72F7727F8E000
:104E5000E69520F4130EB41F651F7A1F330F441F0D
:104E6000551FAA1FFA95A1F7F82F8827F69520F469
:104E7000B40F651F7A1F8E1F440F551FAA1FEE1F08
:104E8000FF23A1F788231AF4939539F418CF000C67
:104E9000111CBB1F661F771F881F012808959F9351
:104EA0009F77993358F050E449EC3FE02BED97DEC3
:104EB0005FEB49EC3FE02BEDA6DDC6DE5F9150785D
:104EC000952708951F930F930027192F10789F7728
:104ED0005FE340E8613071058407950710F00068D2
:104EE00009DE912B6F937F938F939F9386DFEAE187
:104EF000FFE4E8DE5F914F913F912F9182DF002325
:104F000049F02BED3FE049EC5FE300E8902717FD07
:104F1000506879DD0F911F91089508763BD74A7943
:104F2000846E027A2FC1FE7B9A31747B5A3D837C5A
:104F3000917FC77C4CBBE57DAAAA6C7F0000000076
:104F400055914591359125910895991B79E004C0BB
:104F5000991F961708F0961B881F7A95C9F78095B8
:104F6000089597FB092E07260AD077FD04D00CD0B0
:104F700006D000201AF4709561957F4F0895F6F7DA
:104F8000909581959F4F0895AA1BBB1B51E107C0C7
:104F9000AA1FBB1FA617B70710F0A61BB70B881FC9
:104FA000991F5A95A9F780959095BC01CD01089558
:104FB00085FD17C080629923A1F4813694F08B3768
:104FC00084F40895082E806281361CF087364CF4F4
:104FD0000895802D09C08F93EDDF8F9109F08F7DAB
:104FE00008959927882708959923D9F78033CCF31A
:084FF0008A33BCF70895FFCFDE
:00000001FF
